:1000000078C09EC056C39CC09BC0A3C099C098C076
:1000100097C096C095C094C037C192C091C09A4510
:10002000A046A647AD48B349B960BF61C562CB637E
:10003000D164D765DD66E367E968EF69F580FB8128
:10004000FF82FF83FF84FF84FF84FF210101010100
:1000500002030406090E162338596A7F97B4D6FFA7
:100060001400081400080E140004080E1400030500
:10007000080E140004080B0E1114000305080B0EE3
:100080001014000305080B0E1012140008000E00D7
:10009000080E0004080E000305080E0004080E11E7
:1000A00000080E1100F3F404080E10121400080AE0
:1000B0000C0E0F10121400080EED140004050607B4
:1000C00000041400040E1400040810140004080FA7
:1000D0001114000305080A0E0004080B0E00EEEDD3
:1000E000ECEB140E08040004080E00EBECEDEEF34C
:1000F000F41411241FBECFE5D1E0DEBFCDBF20E058
:10010000A0E6B0E001C01D92A937B207E1F7EAE727
:10011000F0E085E5808781E0838314821282868304
:1001200011828BE0818788E58287E0E6F0E08DEF41
:1001300087838EEF8583712C55245A94A6D0D4C220
:100140005FCF8150E82FF0E0E45BFF4FE491EBBD1F
:100150000895189525B7277E25BF29B7226029BFA6
:1001600021E022BF019728F020E188952150E9F78E
:10017000F9CF089588EE93E0EDCF369A3699FECF09
:1001800085B10895CF93C72D81E0870D8F73782EA9
:10019000662D90E09BD26FEF8C2F90E0CF9196C2AE
:1001A000FF920F931F93CF93DF93F82E0BE710E08E
:1001B000CEE7D0E0F11005C0CE0180D2F8018083F7
:1001C00004C0F8016081CE0181D221970F5F1F4FDB
:1001D000C437D10579F7DF91CF911F910F91FF902F
:1001E0000895D0DF81E0DCCF811102C01BBC0895EF
:1001F000A8CF0F931F93CF93C82F8B01CC2359F017
:1002000085E09FDFC801A6DF1BBCC801A3DFC801D2
:10021000A1DFC150F3CFCF911F910F910895EF92BD
:10022000FF920F931F93CF93C8E0E82EF12C062F77
:1002300010E084E186DFC7018DDF1BBCC8018ADFC7
:10024000C150B9F7CF911F910F91FF90EF90089592
:100250001F93CF93DF938FEA87B986EC86B910E1BD
:10026000C0E0D0E085E090E075DF87DFC80FD11DEA
:100270001150C1F7CE0124E0969587952A95E1F7B4
:10028000DF91CF911F91089518951092790087E71B
:1002900090E014D2853519F0612CA3DF11C0712CC8
:1002A000872D90E00BD2682E8F3F19F080E078DF29
:1002B00007C0872D91E0970D792E803488F3F6CF13
:1002C00020918300C0917D0010917E0080917B0081
:1002D000882319F010E0C0E02AE12F5F90E040E0B1
:1002E00050E0A0E6B0E0222379F0BD016F5F7F4FC0
:1002F000FB013197E491EE2319F0962F9A1BF6CF6C
:100300002150AD01DB01EFCF092F6C2F70E0A92F39
:10031000B0E0E02FF0E0112321F09D012E1B3F0BF8
:1003200005C09F0121503109260F371F3197E40F77
:10033000F51FF49027593F4FF901F082015049F71A
:100340009C0F90938500CC2371F0112329F0292F65
:1003500030E02150310902C020E030E0F901E759D6
:10036000FF4F41E0408327E0290F322F3150E32F28
:10037000E91BF0E0E551FF4FE491A32FB0E0A7594E
:10038000BF4FEC933913F2CFE22FF0E0E859FF4F63
:1003900031E0509169004081541330E0231B2093D9
:1003A0008600362D353FE8F5452D4330B0F4809179
:1003B00087008F3F29F4809179008093870006C0E1
:1003C00081E0860D682E891708F0612C80918700E6
:1003D0008F5F8F718093870024C0309179003093B4
:1003E00087004730C0F430918000332311F0882318
:1003F00039F081E0860D682E891798F0612C11C0C4
:10040000862D6916D9F3662019F08150682E09C02F
:100410002150622E06C08111F1CF80917C0088238B
:1004200069F3512C8FEF8DBD80E68CBDAA9A8FE3C6
:1004300084BB83E187BB88EE88BB81E083BF8ABD34
:1004400080BF8BB780628BBF8AB785608ABF85B754
:10045000806285BF789481E287B986EC86B9369947
:10046000FECFC62DC53F10F0612C3CC080918700A7
:10047000803138F4E62DF0E0E759FF4FC081DC2FE2
:1004800031C078DE8091790080938700CBE7D0E09F
:1004900000E010E0FF24F39481E0800F0F5F1F4F16
:1004A00098819F3F29F4219608301105A9F7E2CFE2
:1004B0006DE570E09EDEF801E05AFF4F60808881B4
:1004C0008F2588838EDE6FE070E080E292DE888187
:1004D0008F258883612C85DE4DDE80917B0088230B
:1004E00011F3C8CF4FDE10E0F12C81E2E82E96EC3C
:1004F000D92ECC24CA94CE3E19F463E481E204C020
:10050000CD3E21F468E284E18ADE74C0CC3E11F471
:1005100069E203C0CB3E19F462E581E0F5CFC33F49
:1005200081F404E084E10DDE85E090E013DE88E0F4
:1005300008DE81E490E00EDE0150A1F780ED92E04C
:1005400058C0C43F51F584E690E004DE16DE90E02A
:10055000292F30E0F901E25EFF4FE491E81710F433
:100560009E5FF6CFF901E15EFF4F04916DE770E009
:10057000802F8295869587703CDE8EEE92E0EADDD4
:1005800065E070E081E035DE85E694E0E3DD6DE76F
:1005900070E0802F8F712DDE0DC0CE3F71F400E032
:1005A000009383001EDE6AEF70E081E022DE0F5FC1
:1005B0000A31B1F7DFDDDEDD1DC0CD3F59F58FEF2C
:1005C000809384000EDE85E0BCDDD4DDD3DD84E1E4
:1005D000B8DD3EDE8093840004DECCDDCBDDF9CFD8
:1005E0003699FECFF394909184008917C8F484EF74
:1005F00091E0B0DD8091790080938700BEDD8D3A77
:1006000098F51F5F183008F476CFD53190F010E0E0
:10061000DAE0CAE08D2FE8DD1BDEE7B8D6B8E0CF20
:10062000D93028F3F4E1FF1510F7C0927900D8E033
:10063000DECFD23030F08D2F86958695D695D80FA7
:1006400012C01BBC85B7877E806185BFF89485B7D3
:10065000846885BF8B7F85BF85B7806285BF88959D
:1006600085B78F7D85BFCD2F10E045CF112416B8FB
:100670001BBC87B38C7E87BB94E4B29914C053949F
:10068000999885B7877E806185BFA89591BD85B70C
:10069000846885BF8B7F85BF78948895F89481B5F1
:1006A0008F7B81BDEACF8FE58DBF81E08EBF1FBEFE
:1006B000ECDD552011F0189501C0D8DFE199FECF8F
:1006C0001FBA8EBBE09A99278DB30895262FE19922
:1006D000FECF1CBA1FBA8EBB2DBB0FB6F894E29AA0
:0C06E000E19A0FBE01960895F894FFCF38
